:020000040000FA
:10000000000083160313880183309F0083120313BB
:10001000880141309F009E20102018205E200C286F
:100020000730B000B00B12281F151F191528080043
:100030001E08B100831603131E0883120313B200B7
:100040000310B20D031C25280314B10D0310B20DCB
:10005000031C2B280314B10DB301B401B501B60183
:10006000B108031947280314E830B20203183928ED
:10007000B10303140330B10203184528B10703107C
:10008000E830B2070318B10A4728B30A30286430B1
:100090000314B20203185028B10803195228B103FF
:1000A000B40A4728B2070A300314B202031C5A28C4
:1000B000B50A5328B2073208B6000800F4108030A1
:1000C0008E20F4143030B307B407B507B6073308F1
:1000D0008E202E308E2034088E2035088E20360853
:1000E0008E2020308E2056308E206F308E206C3047
:1000F0008E2074308E2073308E200800F930F0008E
:100100000000F00B80280800F1007E20F10B85280C
:10011000080008157E2008117E200800F500F0393F
:100120008800F418881489207E20F50E7508F039AF
:100130008800F418881489207E2008006430842008
:10014000F030F40030308800892005308420892088
:100150007E2089200812892028308E2008308E20A9
:1001600001308E2006308E2080308E200C308E2084
:02017000080085
:02400E00313748
:00000001FF
